:020000040000FA
:020000000528D1
:06000A008312850183163C
:10001000FE30850061308F001A309F0083128312FA
:10002000073099000D309F000510003090000C1033
:10003000FE308F00D4308E001014C0200130270213
:10004000031D2328322802302702031D28283228C6
:1000500003302702031D2D28322804302702031DF8
:10006000152883289F151F15ED201E08A3000310D7
:10007000A30C9F151F11ED201E08A200851A45280C
:100080000530A202031CA2014D2885194D28053018
:10009000A207031C4D28FF30A2002208A100013056
:1000A0002702031D54285E2802302702031D592809
:1000B000632803302702031D152868283E21A50068
:1000C0004A22A6006C285623A5006224A6006C28AC
:1000D0006E25A5007A26A6000C1C6C282030900006
:1000E0000C1025088F0026088E0010140514CC2053
:1000F000A30803197F280000A30B7B28000005102C
:100100000C1C80281528DC20C02004302702031D89
:100110001528AF202B1884289F151F11ED201E08CD
:10012000A4009F151F15ED201E08A300A4080319A5
:100130009C28D320A40B99280514CC20A3080319CC
:10014000A5280000A30BA12800000510C020043042
:100150002702031D1528AF202B1CA6288328A901E0
:100160000A30AA00851EB528A90AAA0BB2282908B8
:10017000053C031CBD282B10BF282B1400000800D1
:100180009F111F15ED201E08A1000310A10C0310E4
:10019000A10CF220A70008000B30A8000000A80B5B
:1001A000CE2800000800EA30A8000000A80BD528DF
:1001B00000000000000008003030A8000000A80B7C
:1001C000DE2800000000000008000430A800A80B92
:1001D000E7280000000000000800E5209F149F1899
:1001E000EF2808002108A000FE30A0070030031807
:1001F000013E8A002008FD200800820000340034FF
:100200000034FF34FF34FF34FF34FF34FF34FF3455
:10021000FF34FF34013401340134FF34FF34FF3440
:100220000234023402340234FF34FF340334033422
:1002300003340334FF34FF3404340434043404340A
:100240000434FF34FF34FF34FF34FF34FF34FF3411
:10025000FF34FF34FF34FF34FF34FF34FF34FF3406
:10026000FF34FF34FF34FF34FF34FF34FF34FF34F6
:10027000FF34FF34FF34FF34FF34FF342108A00083
:100280004A30A00701300318013E8A0020084921A6
:10029000080082003C343E3440344134423444341B
:1002A00045344734483449344B344C344D344F345E
:1002B00050345134523453345534563457345834FE
:1002C00059345A345B345C345D345F3460346134A7
:1002D0006234633464346534653466346734683456
:1002E00069346A346B346C346D346E346E346F340C
:1002F00070347134723473347334743475347634C6
:10030000763477347834793479347A347B347C3485
:100310007C347D347E347E347F3480348034813448
:10032000823482348334833484348534853486340F
:100330008634873488348834893489348A348A34DA
:100340008B348C348C348D348D348E348E348F34A5
:100350008F34903490349134913492349234933475
:100360009334943494349534953495349634963447
:1003700097349734983498349934993499349A341A
:100380009A349B349B349B349C349C349D349D34F0
:100390009D349E349E349F349F349F34A034A034C7
:1003A000A034A134A134A134A234A234A334A334A0
:1003B000A334A434A434A434A534A534A534A63479
:1003C000A634A634A734A734A734A734A834A83455
:1003D000A834A934A934A934AA34AA34AA34AA3432
:1003E000AB34AB34AB34AC34AC34AC34AC34AD340F
:1003F000AD34AD34AE34AE34AE34AE34AF34AF34ED
:10040000AF34AF34B034B034B034B034B134B134CC
:10041000B134B134B234B234B234B234B334B334AC
:10042000B334B334B434B434B434B434B534B5348C
:10043000B534B534B534B634B634B634B634B6346F
:10044000B734B734B734B734B834B834B834B83450
:10045000B834B934B934B934B934B934BA34BA3433
:10046000BA34BA34BA34BB34BB34BB34BB34BB3417
:10047000BC34BC34BC34BC34BC34BC34BD34BD34FA
:10048000BD34BD34BD34BD34BE34BE34BE34BE34E0
:10049000BE34BF342108A0005630A0070230031834
:1004A000013E8A002008552208008200FF34833470
:1004B00001347934EB345734BE3420347D34D434B1
:1004C00027347434BD34013441347C34B334E634DD
:1004D00014343E3464348634A534BF34D634E9341D
:1004E000F93405340E341334153414340F3408340D
:1004F000FD34F034DF34CC34B5349C348034623491
:1005000040341D34F634CD34A234743444341134C0
:10051000DC34A5346C343034F334B33471342D34DA
:10052000E7349F3455340934BB346C341A34C7343F
:1005300072341B34C23468340C34AF344F34EF346B
:100540008C342834C3345C34F4348A341E34B134EB
:100550004334D4346334F1347D34083492341A345F
:10056000A2342834AD343034B3343434B434333476
:10057000B1342E34A93424349D3416348D340434EB
:100580007934ED346134D3344534B534253493347F
:1005900001346E34DA344534AF3419348134E934FB
:1005A0004F34B5341B347F34E3344534A734093435
:1005B0006934C93428348634E43441349D34F93400
:1005C0005334AD3407346034B8340F346634BC343B
:1005D00012346734BB340F346234B43406345834C4
:1005E000A834F93448349734E63434348134CE3482
:1005F0001B346634B234FC3447349134DA34233457
:100600006B34B334FA3441348734CD341334583432
:100610009C34E13424346834AA34ED342F347034FB
:10062000B134F23432347234B234F1342F346E34A3
:10063000AC34E93426346334A034DC341734533416
:100640008E34C83402343C347634AF34E834203449
:1006500059349034C834FF3436346D34A334D9342B
:100660000E3444347934AD34E23416344A347D34B3
:10067000B034E334163448347A34AC34DE340F34D6
:1006800040347134A134D1340134313460348F3486
:10069000BE34ED341B3449347734A534D234FF34BE
:1006A0002C3459348534B234DE3409342108A000A6
:1006B0006230A00703300318013E8A00200861233E
:1006C00008008200BF34BF34BF34BF34C034C034EC
:1006D000C034C034C134C134C134C134C234C23472
:1006E000C234C234C334C334C334C334C334C43453
:1006F000C434C434C434C534C534C534C534C53435
:10070000C634C634C634C634C634C734C734C73416
:10071000C734C734C834C834C834C834C834C834FB
:10072000C934C934C934C934C934CA34CA34CA34DE
:10073000CA34CA34CA34CB34CB34CB34CB34CB34C4
:10074000CB34CC34CC34CC34CC34CC34CC34CD34A9
:10075000CD34CD34CD34CD34CD34CD34CE34CE348F
:10076000CE34CE34CE34CE34CF34CF34CF34CF3475
:10077000CF34CF34CF34D034D034D034D034D0345C
:10078000D034D034D034D134D134D134D134D13444
:10079000D134D134D234D234D234D234D234D2342B
:1007A000D234D234D334D334D334D334D334D33413
:1007B000D334D334D334D434D434D434D434D434FC
:1007C000D434D434D434D534D534D534D534D534E4
:1007D000D534D534D534D534D634D634D634D634CD
:1007E000D634D634D634D634D634D634D734D734B7
:1007F000D734D734D734D734D734D734D734D734A1
:10080000D834D834D834D834D834D834D834D83488
:10081000D834D834D934D934D934D934D934D93472
:10082000D934D934D934D934D934D934DA34DA345E
:10083000DA34DA34DA34DA34DA34DA34DA34DA3448
:10084000DA34DB34DB34DB34DB34DB34DB34DB3431
:10085000DB34DB34DB34DB34DB34DC34DC34DC341D
:10086000DC34DC34DC34DC34DC34DC34DC34DC3408
:10087000DC34DC34DD34DD34DD34DD34DD34DD34F2
:10088000DD34DD34DD34DD34DD34DD34DD34DD34E0
:10089000DE34DE34DE34DE34DE34DE34DE34DE34C8
:1008A000DE34DE34DE34DE34DE34DE34DE34DF34B7
:1008B000DF34DF34DF34DF34DF34DF34DF34DF34A0
:1008C000DF34DF342108A0006E30A00704300318A5
:1008D000013E8A0020086D240800820035347634F9
:1008E000B634F63435347434B334F0342E346B34D7
:1008F000A734E3341F345A349534CF3409344334A5
:100900007C34B434ED3424345C349334C93400344E
:1009100035346B34A034D53409343D347134A434C7
:10092000D73409343C346D349F34D03401343234FC
:1009300062349234C134F1341F344E347C34AA34DE
:10094000D8340634333460348C34B834E43410345E
:100950003B3467349134BC34E63410343A34643474
:100960008D34B634DF340734303458347F34A73410
:10097000CE34F5341C34433469348F34B534DB342D
:10098000003425344A346F349434B834DC340034C1
:10099000243448346B348E34B134D434F6341934BE
:1009A0003B345D347E34A034C134E3340434243425
:1009B000453466348634A634C634E63405342534EA
:1009C000443463348234A134BF34DE34FC341A340A
:1009D0003834563473349134AE34CB34E83405347F
:1009E00022343F345B3477349334AF34CB34E73440
:1009F00002341E34393454346F348A34A534BF344D
:100A0000DA34F4340E34293442345C34763490349D
:100A1000A934C234DC34F5340E3426343F3458342F
:100A200070348934A134B934D134E9340134183400
:100A3000303447345F3476348D34A434BB34D2340C
:100A4000E834FF3416342C34423458346F3485344F
:100A50009A34B034C634DB34F13406341C343134C7
:100A600046345B34703485349A34AE34C334D7346E
:100A7000EC340034143428343C3450346434783446
:100A80008C349F34B334C634D934ED340034133449
:100A9000263439344C345F34713484349734A93477
:100AA000BB34CE34E034F2340434163428343A34CF
:100AB0004C345E346F3481349334A434B534C73449
:100AC000D834E934FA340B341C342D343E344F34EA
:100AD0005F34703481349134A134B2342108A000E1
:100AE0007A30A00705300318013E8A0020087925D6
:100AF00008008200DF34DF34DF34E034E034E034F7
:100B0000E034E034E034E034E034E034E034E03445
:100B1000E034E034E134E134E134E134E134E1342F
:100B2000E134E134E134E134E134E134E134E2341C
:100B3000E234E234E234E234E234E234E234E23405
:100B4000E234E234E234E234E234E334E334E334F2
:100B5000E334E334E334E334E334E334E334E334DD
:100B6000E334E334E334E334E434E434E434E434C9
:100B7000E434E434E434E434E434E434E434E434B5
:100B8000E434E434E434E434E534E534E534E534A1
:100B9000E534E534E534E534E534E534E534E5348D
:100BA000E534E534E534E534E534E534E634E6347B
:100BB000E634E634E634E634E634E634E634E63465
:100BC000E634E634E634E634E634E634E634E63455
:100BD000E734E734E734E734E734E734E734E7343D
:100BE000E734E734E734E734E734E734E734E7342D
:100BF000E734E734E734E734E734E834E834E8341A
:100C0000E834E834E834E834E834E834E834E83404
:100C1000E834E834E834E834E834E834E834E834F4
:100C2000E834E834E834E934E934E934E934E934DF
:100C3000E934E934E934E934E934E934E934E934CC
:100C4000E934E934E934E934E934E934E934E934BC
:100C5000E934E934E934EA34EA34EA34EA34EA34A7
:100C6000EA34EA34EA34EA34EA34EA34EA34EA3494
:100C7000EA34EA34EA34EA34EA34EA34EA34EA3484
:100C8000EA34EA34EA34EA34EA34EB34EB34EB3471
:100C9000EB34EB34EB34EB34EB34EB34EB34EB345C
:100CA000EB34EB34EB34EB34EB34EB34EB34EB344C
:100CB000EB34EB34EB34EB34EB34EB34EB34EB343C
:100CC000EB34EB34EC34EC34EC34EC34EC34EC3426
:100CD000EC34EC34EC34EC34EC34EC34EC34EC3414
:100CE000EC34EC34EC34EC34EC34EC34EC34EC3404
:100CF000EC34EC342108A0008630A007063003183D
:100D0000013E8A002008852608008200C234D834BB
:100D1000ED34033418342D34423457346C34813478
:100D20009634AA34BF34D334E734FB340F3423343D
:100D300037344B345F34723486349934AC34C03435
:100D4000D334E634F9340B341E343134433456345E
:100D500068347A348C349F34B134C234D434E634B9
:100D6000F83409341B342C343E344F34603471343D
:100D700082349334A434B534C634D634E734F734EB
:100D800008341834283438344934593469347934BF
:100D900088349834A834B734C734D734E634F534BB
:100DA0000534143423343234413450345F346E34D7
:100DB0007D348B349A34A834B734C534D434E23417
:100DC000F034FF340D341B34293437344534533474
:100DD00060346E347C348A349734A534B234C034F1
:100DE000CD34DA34E734F53402340F341C3429348A
:100DF000363443344F345C346934763482348F343F
:100E00009B34A834B434C134CD34D934E534F2340D
:100E1000FE340A34163422342E343A3446345134F3
:100E20005D346934753480348C349734A334AE34F3
:100E3000BA34C534D034DC34E734F234FD34083409
:100E400014341F342A3435343F344A345534603432
:100E50006B34753480348B349534A034AA34B53473
:100E6000BF34CA34D434DE34E934F334FD340734C7
:100E700012341C34263430343A3444344E3458342A
:100E800061346B3475347F34893492349C34A634A5
:100E9000AF34B934C234CC34D534DF34E834F1342F
:100EA000FB3404340D3417342034293432343B34C9
:100EB00044344D3456345F34683471347A34833476
:100EC0008C3495349D34A634AF34B834C034C9342E
:100ED000D234DA34E334EB34F434FC3405340D34F6
:100EE00016341E3426342F3437343F3447344F34CD
:100EF00058346034683470347834803488349034B2
:0C0F00009834A034A834B034B834C034A5
:02400E00C430BC
:00000001FF
